:020000000C28CA
:10000800FE00030EF4000408F5000A08F600402D6F
:10001800BF2E43278326DE01BF01C001B42BFF306A
:10002800AB01AC003F08F726003A0319B42BBF0A0E
:100038002E283F08FF3EAB00FF30AC01AD003F0863
:100048004326003A0319B42B3F08073A031D30280A
:100058000630BF00DE0AB42BBF0AB42B3F0AAB0040
:10006800FF30AC01AD003F084326003A0319B42B1A
:10007800BF0803192E28BF03B42BFF30AB00003094
:10008800AC01F726003A0319B42BBF012E283F080C
:10009800073CAB00FF30AC01AD003F086326003AD7
:1000A8000319B42B3F08033AD1283F08073CAB009B
:1000B800FF30AC00AD013F086326003A0319B42BAA
:1000C8003F08033A031D302803302D283F08073C1A
:1000D800AB00FF30AC01AD003F086326003A0319BE
:1000E800B42BBF08031968283F283F08073CAB001A
:1000F800FF30AC00AD013F086326003A0319B42B6A
:10010800BF08031D3F28BF01DE0A1128FF30AB00DE
:100118000030FE257E2BFF30AB01FE25003A031987
:10012800B42B4008053A03192E28DE03C00AB42B65
:100138000330AB000530AC000730AD00FF30AE0037
:100148000130AF01D425003A0319B42B302BFF300E
:10015800AB01AC003F08F726003A0319B42B3F085F
:10016800023AD1283F08033EAB00FF30AC00AD0196
:100178003F084326003A0319B42B3F08043A031DED
:10018800302805302D28FF30AB00AC013F08F7269A
:10019800003A0319B42B3F08073A031949283028B5
:1001A800BC01FF30A8003C0890273C08BB000310A6
:1001B800BB0D03103B0DA03E84000008A300840A79
:1001C8000008A400840A0008A500840A0008A60004
:1001D800DB26A8013C0890270830BC0A3C02031C17
:1001E800D5280630BC00FF30A8003C0890273C0802
:1001F800BB000310BB0D03103B0DA03E840000089C
:10020800A300840A0008A400840A0008A500840A40
:100218000008A600DB26A8013C089027BC0BF7289D
:10022800FF30A8003C0890273C08BB000310BB0D1A
:1002380003103B0DA03E84000008A300840A0008B8
:10024800A400840A0008A500840A0008A600DB268A
:10025800A8013C089027DE0A0730BD00FF30A8003F
:100268003D089027FC30A0003D086527BC3E84006F
:100278000008A300840A0008A400840A0008A50056
:10028800840A0008A600DB26A8013D089027BD0BBC
:100298003229FF30A8003D089027FC30A0003D0817
:1002A8006527BC3E84000008A300840A0008A40057
:1002B800840A0008A500840A0008A600DB26A80115
:1002C8003D089027BD01BD0AFF30A8003D089027D2
:1002D800FC30A0003D086527BC3E84000008A30050
:1002E800840A0008A400840A0008A500840A0008FB
:1002F800A600DB26A8013D0890270830BD0A3D026C
:1003080003182E286829BE0108303E020318BC29AC
:10031800FF30A8003E089027FF30A8003E08073CA1
:10032800902704303E020318A1293E08BB000310A1
:10033800BB0D03103B0DA03EA629FC30A0003E08D3
:100348006527BC3E84000008A300840A0008A400B6
:10035800840A0008A500840A0008A600DB26A80174
:100368003E089027A8013E08073C9027BE0A882926
:10037800BE0104303E0203182E2804303E02031842
:10038800EA293E08A000A101A00A0319A10AFF302A
:10039800A200A3018F252008A8003E0890273E0848
:1003A800A000A101A00A0319A10AFF30A200A3011D
:1003B8008F252008A8003E08073C90273E08BB0070
:1003C8000310BB0D03103B0DA03E0E2A0830A00001
:1003D800A1013E08A002031CA103FF30A200A30153
:1003E8008F252008A8003E0890270830A000A1010A
:1003F8003E08A002031CA103FF30A200A3018F2521
:100408002008A8003E08073C9027FC30A0003E08C2
:100418006527BC3E84000008A300840A0008A400E5
:10042800840A0008A500840A0008A600DB26A801A3
:100438003E089027A8013E08073C9027BE0ABD2920
:100448000430AB00FF30AC000330AD0163267E2BD7
:100458003230E000FF30E101AB01AC003F08F72685
:100468007E2BC008031D3C2A2030E00003305B2AA5
:10047800400B402ABC30452A4008023A031D482A4E
:100488005830E00002305B2A4008033A031D4E2A28
:10049800F430592A4008043A031D542A9030592A46
:1004A8004008053A031D5D2A2C30E0000130E100C8
:1004B800BC2A4008063A031D632AC830BA2A4008F5
:1004C800073A031D692A6430BA2A4008083A031D0E
:1004D8006F2A5030BA2A4008093A03196D2A400891
:1004E8000A3A031D792A4630BA2A40080B3A031DF6
:1004F8007F2A3C30BA2A40080C3A031D852A32303C
:10050800BA2A40080D3A031D8B2A2830BA2A400817
:100518000E3A031D912A1E30BA2A40080F3A031DCD
:10052800972A1430BA2A4008103A031D9D2A0A3027
:10053800BA2A4008113A031DA32A0930BA2A4008EA
:10054800123A031DA92A0830BA2A4008133A031D93
:10055800AF2A0730BA2A4008143A031DB52A0630D4
:10056800BA2A4008153A031DBC2A0530E000E1010B
:10057800FF30AB00AC013F08F726003A0319B42B53
:10058800C00A400BCB2A0330BF00DE03B42B40085F
:10059800023A031DD12A0730C82A4008033A031D2E
:1005A800D72A0230C82A4008043A031DDD2A05303C
:1005B800C82A4008053A031DE42ABF01BF0AC92A10
:1005C8004008063A031DEA2A0430C82A4008073AB8
:1005D800031DF02A0630C82A4008083A0319C72A1A
:1005E8004008093A0319CF2A40080A3A0319D52ABC
:1005F80040080B3A0319DB2A40080C3A0319E12A90
:1006080040080D3A0319E82A40080E3A0319EE2A61
:1006180040080F3A0319C72A4008103A0319CF2A8D
:100628004008113A0319D52A4008123A0319DB2A5F
:100638004008133A0319E12A4008143A0319E82A32
:100648004008153A0319EE2A4008163A031DB42B40
:10065800F430E0000130E100BF01C0012E280A306B
:10066800A800003090270A30A800013090270A30EF
:10067800A800023090270A30A800033090270A30DB
:10068800A800043090270A30A800053090270A30C7
:10069800A800063090270A30A80007309027FF30BE
:1006A800AB0000309324003A0319B42B1F30A60185
:1006B800A500FF30A400A300DB262E280030AB01E4
:1006C800ED24003A0319B42BC030E2005D30E3009A
:1006D8002E282830AB01AC001430AD01AE000A3032
:1006E800AF01B0002730B101B200FF30B301B4014F
:1006F800B5013024003A031D2E28B42B2830AB0056
:100708001430AC01AD000A30AE01AF00FF30B001CB
:10071800B1002730B2000030B301B401B501C023E5
:10072800003A0319B42B0030A80190270130A80122
:1007380090270230A80190270330A80190270430A1
:10074800A80190270530A80190270630A801902716
:100758000730A8019027F430E2000130E300DE0101
:100768005E088400183004020318B42B07308A008E
:100778002B30040782000C28B700B801DF08031DDE
:10078800D72B3708C9002B08CA002C08CB002D0826
:10079800CC002E08CD002F08CE003008CF0031083D
:1007A800D000DF01DF0A4908C1004A08C2004B082F
:1007B800C3004C08C4004D08C5004E08C6004F08C9
:1007C800C7005008C800BA015D083A02B900B91F4D
:1007D800F12B3A082924493EF42B3A082924413EB2
:1007E8008400360880000830BA0A3A02031CE82B55
:1007F800DD0A5D08803A783E0318DD01D90A03193D
:10080800DA0A0319DB0A0319DC0A5C083502031D3E
:10081800172C5B083402031D172C5A083302031DDA
:10082800172C590832020318202CDF01B801B80A26
:10083800D901DA01DB01DC016208A3006308A40026
:10084800A501A601DB2638080800493E8400831369
:100858000008B60039080800B700B801DF08031D12
:10086800482C3708C9002B08CA002C08CB002D08D3
:10087800CC002E08CD002F08CE003008CF0031085C
:10088800D000DD01DF01DF0ABA013A085D07B900CF
:10089800083039023A08031C552C493E8D24393E4C
:1008A800582C493E8D24413E84003608800008308B
:1008B800BA0A3A02031C492CDD0A5D08803A783EE0
:1008C8000318DD01D90A0319DA0A0319DB0A031927
:1008D800DC0A5C083502031D7B2C5B083402031D0F
:1008E8007B2C5A083302031D7B2C5908320203184B
:1008F800842CDF01B801B80AD901DA01DB01DC0177
:100908006208A3006308A400A501A601DB26380835
:100918000800840083130008B60039080800AC00FA
:10092800AD01DF08031DAA2C4108C9004208CA000E
:100938004308CB004408CC004508CD004608CE004B
:100948004708CF004808D000DF01DF0A4908C10086
:100958004A08C2004B08C3004C08C4004D08C50033
:100968004E08C6004F08C7005008C8004908FF3A9B
:10097800031DC90A4A08FF3A031DCA0A4B08FF3A71
:10098800031DCB0A4C08FF3A031DCC0A4D08FF3A59
:10099800031DCD0A4E08FF3A031DCE0A4F08FF3A41
:1009A800031DCF0A5008FF3A031DD00A2C08493E00
:1009B800840000082B06031DE42CDF01AD01AD0AFD
:1009C8006208A3006308A400A501A601DB262D0880
:1009D8000800AC00AD01DF08031D042D4108C90063
:1009E8004208CA004308CB004408CC004508CD00A3
:1009F8004608CE004708CF004808D000DF01DF0ACC
:100A08004908C1004A08C2004B08C3004C08C4008A
:100A18004D08C5004E08C6004F08C7005008C8005A
:100A28004908031DC9034A08031DCA034B08031DCF
:100A3800CB034C08031DCC034D08031DCD034E0802
:100A4800031DCE034F08031DCF035008031DD00319
:100A58002C08493E8400831300082B06031D372DFC
:100A6800DF01AD01AD0A6208A3006308A400A50177
:100A7800A601DB262D0808000B198B1E862D77088A
:100A8800413E84008313000878020318642D770818
:100A9800513E84008008031D7C2D0130F300770A45
:100AA800572D0310F30DFF3E031D552D7308F90450
:100AB8007908A1267708513E8400013080007C2DFA
:100AC8007708513E8400800803197C2D0130F3001B
:100AD800770A702D0310F30DFF3E031D6E2D73086A
:100AE800FF3AF9057908A1267708513E840080016C
:100AF800F80AF70A083077020318F701A0300B113B
:100B08008312810076088A0075088400740E8300B9
:100B1800FE0E7E0E0900A501A11F992DA009A109AD
:100B2800A00A0319A10AA501A50AA31FA22DA209BB
:100B3800A309A20A0319A30A0130A506A601A70161
:100B4800210820040319C72DA401A40AA11BB02D54
:100B58000310A00DA10DA92D0310A60DA70D2108A6
:100B68002302031DB92D20082202031CC32D2008CF
:100B7800A2022108031CA303A30226140310A10C3C
:100B8800A00CA40BB02D25080319CF2DA609A70981
:100B9800A60A0319A70A2708A1002608A00008002A
:100BA800B000B1012F08A3002E0873273008413E7A
:100BB80084004908831380002B08413E84004908BB
:100BC80080002C08413E8400490880002D08413EE1
:100BD8008400490880000130A601A501A400F43072
:100BE800A300DB265F30A0003130A1002F081227B8
:100BF80031080800AC00AD012B08A3002C087327AE
:100C08004908C1004908C3004908C5004908C70088
:100C18004909C2004909C4004909C6004909C80070
:100C28000130A601A501A400F430A300DB265F3043
:100C3800A0002D30A1002B0812272D0808005034E1
:100C4800C3340034003420344E340034003430349B
:100C58007534003400345034463400340034803461
:100C68003E3400340034B034363400340034E034D8
:100C78002E34003400341034273400340034AE00ED
:100C8800AF012D08A3002C0873272E08413E8400CD
:100C98004908831380002B08413E840049098000DD
:100CA8000130A601A501A400F430A300DB265F30C3
:100CB800A0002F30A1002D0812272F080800AE0031
:100CC800AF012D08A3002C0873272E08413E84008D
:100CD8004908831380002B08413E8400490880009E
:100CE8000130A601A501A400F430A300DB265F3083
:100CF800A0002F30A1002D0812272F080800831606
:100D08008F150F10011081100111811581120B111F
:100D18008B168B170B178312C101C201C301C401C3
:100D2800C501C601C701C801D101D201D301D4014F
:100D3800D501D601D701D8010800F100F2017108E8
:100D4800F000720AA92E0310F00CFF3E031DA72E17
:100D5800701CB12E83128514B32E831285100830AF
:100D6800051005140510F20A7202031CA32E0511C2
:100D78000515051108004130F701F801F901831341
:100D8800840060308027C030FD000630FE0023302C
:100D9800FF00A03084005A27F430E0000130E10061
:100DA800F430E2000130E300E40083010D28A701DC
:100DB800A801A901AA012A082602031DED2E290867
:100DC8002502031DED2E28082402031DED2E2708F9
:100DD8002302031C0800A70A0319A80A0319A90A71
:100DE8000319AA0ADF2EAD00AE012C08A3002B08B8
:100DF80073272D08413E840049088313800060084A
:100E0800A3006108A400A501A601DB265F30A000AD
:100E18002E30A1002C0812272E080800A200640812
:100E28000319252F2208490203181C2FC90A080094
:100E38002008840083138001210884008001800A2F
:100E480008004908220203181C2FC90308001328A8
:100E58001D28322841284B2859286A2879288A28A9
:100E68008F289C28AB28B628C728D428302987295A
:100E7800242A2C2A352A332B622B6D2B822B073000
:100E8800990095019F0183169F0181130510851014
:100E98000511831205108514051183169601831216
:100EA800901108007E088A007F088200562780007B
:100EB800840A04087D0603190034FF0A0319FE0A90
:100EC8005A2FA200A10120082218A1070310A00D83
:100ED8000310A20CA208031D672F21080800A40014
:100EE800DF08031D0800C9002308A000240888277C
:100EF800E400DF01DF0A080064008001840A0406B8
:100F0800031900340406812FA10020082102A20140
:100F1800031CA20A22080800A900413E84002808F0
:060F2800831380000800A5
:02400E00E2F0DE
:00000001FF
